 COMPCIE950

 Timestamp is 49d37346 (Wed Apr 01 14:59:34 2009)

 Preferred load address is 10000000

 Start         Length     Name                   Class
 0001:00000000 00000004H .CRT$XCA                CODE
 0001:00000004 00000004H .CRT$XCZ                CODE
 0001:00000008 00000004H .CRT$XIA                CODE
 0001:0000000c 00000004H .CRT$XIZ                CODE
 0001:00000010 00000004H .CRT$XPA                CODE
 0001:00000014 00000004H .CRT$XPZ                CODE
 0001:00000018 00000004H .CRT$XTA                CODE
 0001:0000001c 00000004H .CRT$XTZ                CODE
 0001:00000020 000009b0H .rdata                  CODE
 0001:000009d0 00000027H .rdata$debug            CODE
 0001:00000a00 00000004H .rdata$sxdata           CODE
 0001:00000a04 00006750H .text                   CODE
 0001:00007158 0000003cH .xdata$x                CODE
 0001:00007194 00000028H .idata$2                CODE
 0001:000071bc 00000014H .idata$3                CODE
 0001:000071d0 00000134H .idata$4                CODE
 0001:00007304 00000016H .idata$6                CODE
 0001:00007320 00000135H .edata                  CODE
 0002:00000000 00000134H .idata$5                DATA
 0002:00000134 00000028H .data                   DATA
 0002:0000015c 00000024H .bss                    DATA

  Address         Publics by Value              Rva+Base       Lib:Object

 0000:00000001       ___safe_se_handler_count   00000001     <absolute>
 0001:00000000       ___xc_a                    10001000     corelib0:crt0init.obj
 0001:00000004       ___xc_z                    10001004     corelib0:crt0init.obj
 0001:00000008       ___xi_a                    10001008     corelib0:crt0init.obj
 0001:0000000c       ___xi_z                    1000100c     corelib0:crt0init.obj
 0001:00000010       ___xp_a                    10001010     corelib0:crt0init.obj
 0001:00000014       ___xp_z                    10001014     corelib0:crt0init.obj
 0001:00000018       ___xt_a                    10001018     corelib0:crt0init.obj
 0001:0000001c       ___xt_z                    1000101c     corelib0:crt0init.obj
 0001:0000003c       ??_C@_1BI@BHLBGEOK@?$AAP?$AAr?$AAi?$AAo?$AAr?$AAi?$AAt?$AAy?$AA2?$AA5?$AA6?$AA?$AA@ 1000103c     mddpcie950:mddpcie950.obj
 0001:00000054       ??_C@_1CC@KMPFMANC@?$AAD?$AAe?$AAv?$AAi?$AAc?$AAe?$AAA?$AAr?$AAr?$AAa?$AAy?$AAI?$AAn?$AAd?$AAe?$AAx?$AA?$AA@ 10001054     mddpcie950:mddpcie950.obj
 0001:000000f4       ??_C@_17KACEIPNC@?$AAK?$AAe?$AAy?$AA?$AA@ 100010f4     serpcie950:serpcie950.obj
 0001:00000100       ??_7CSerialPDD@@6B@        10001100     serpcie950:serpcie950.obj
 0001:000001f4       ??_C@_1CC@EKOCNIBB@?$AAC?$AAr?$AAy?$AAs?$AAt?$AAa?$AAl?$AAF?$AAr?$AAe?$AAq?$AAu?$AAe?$AAn?$AAc?$AAy?$AA?$AA@ 100011f4     serpcie950:serpcie950.obj
 0001:00000218       ??_7CMiniThread@@6B@       10001218     serpcie950:serpcie950.obj
 0001:0000021c       ??_7CSerialPDDPowerUpCallback@@6B@ 1000121c     serpcie950:serpcie950.obj
 0001:00000220       ??_7CRegpcie950@@6B@       10001220     pddpcie950:pddpcie950.obj
 0001:00000338       ??_C@_1CM@HIMBKDJM@?$AAL?$AAi?$AAn?$AAe?$AAD?$AAr?$AAi?$AAv?$AAe?$AAr?$AAD?$AAe?$AAl?$AAa?$AAy?$AAP?$AAh?$AAa?$AAs?$AAe?$AAs?$AA?$AA@ 10001338     pddpcie950:pddpcie950.obj
 0001:00000364       ??_C@_1CI@GLAIJPLJ@?$AAL?$AAi?$AAn?$AAe?$AAD?$AAr?$AAi?$AAv?$AAe?$AAr?$AAD?$AAe?$AAl?$AAa?$AAy?$AAB?$AAi?$AAt?$AAs?$AA?$AA@ 10001364     pddpcie950:pddpcie950.obj
 0001:0000038c       ??_C@_1CE@PJBMNJAF@?$AAL?$AAi?$AAn?$AAe?$AAD?$AAr?$AAi?$AAv?$AAe?$AAr?$AAC?$AAo?$AAn?$AAt?$AAr?$AAo?$AAl?$AA?$AA@ 1000138c     pddpcie950:pddpcie950.obj
 0001:000003b0       ??_C@_1CE@BHEKDMEI@?$AAB?$AAa?$AAu?$AAd?$AAr?$AAa?$AAt?$AAe?$AAM?$AAa?$AAp?$AAL?$AAi?$AAs?$AAt?$AAT?$AAo?$AA?$AA@ 100013b0     pddpcie950:pddpcie950.obj
 0001:000003d4       ??_C@_1CI@OJPKJBA@?$AAB?$AAa?$AAu?$AAd?$AAr?$AAa?$AAt?$AAe?$AAM?$AAa?$AAp?$AAL?$AAi?$AAs?$AAt?$AAF?$AAr?$AAo?$AAm?$AA?$AA@ 100013d4     pddpcie950:pddpcie950.obj
 0001:000003fc       ??_C@_1CE@HLGCKFJ@?$AAF?$AAl?$AAo?$AAw?$AAC?$AAt?$AAr?$AAl?$AAH?$AAi?$AAg?$AAh?$AAL?$AAe?$AAv?$AAe?$AAl?$AA?$AA@ 100013fc     pddpcie950:pddpcie950.obj
 0001:00000420       ??_C@_1CC@ELLFOF@?$AAF?$AAl?$AAo?$AAw?$AAC?$AAt?$AAr?$AAl?$AAL?$AAo?$AAw?$AAL?$AAe?$AAv?$AAe?$AAl?$AA?$AA@ 10001420     pddpcie950:pddpcie950.obj
 0001:00000444       ??_C@_1BO@MCGADMLE@?$AAR?$AAx?$AAI?$AAn?$AAt?$AAT?$AAr?$AAi?$AAg?$AAL?$AAe?$AAv?$AAe?$AAl?$AA?$AA@ 10001444     pddpcie950:pddpcie950.obj
 0001:00000464       ??_C@_1BO@ELCCHGIE@?$AAT?$AAx?$AAI?$AAn?$AAt?$AAT?$AAr?$AAi?$AAg?$AAL?$AAe?$AAv?$AAe?$AAl?$AA?$AA@ 10001464     pddpcie950:pddpcie950.obj
 0001:00000484       ??_C@_1BA@BDHDGOBO@?$AAS?$AAy?$AAs?$AAI?$AAn?$AAt?$AAr?$AA?$AA@ 10001484     pddpcie950:pddpcie950.obj
 0001:00000494       ??_C@_1BE@PGPADFAN@?$AAR?$AAe?$AAg?$AAS?$AAt?$AAr?$AAi?$AAd?$AAe?$AA?$AA@ 10001494     pddpcie950:pddpcie950.obj
 0001:000004a8       ??_C@_1BC@DEOLOKPA@?$AA?2?$AAo?$AAp?$AAt?$AAi?$AAo?$AAn?$AA1?$AA?$AA@ 100014a8     pddpcie950:pddpcie950.obj
 0001:000004bc       ??_C@_17DBKELHOO@?$AAP?$AAN?$AAP?$AA?$AA@ 100014bc     pddpcie950:pddpcie950.obj
 0001:000004c4       ??_C@_1BC@NIOILLNH@?$AAI?$AAN?$AAS?$AAT?$AAA?$AAN?$AAC?$AAE?$AA?$AA@ 100014c4     pddpcie950:pddpcie950.obj
 0001:000004d8       ??_C@_1BI@FDNCMLGC@?$AAB?$AAU?$AAI?$AAL?$AAT?$AAI?$AAN?$AA?2?$AAP?$AAC?$AAI?$AA?$AA@ 100014d8     pddpcie950:pddpcie950.obj
 0001:000004f0       ??_7CMemRegpcie950@@6B@    100014f0     pddpcie950:pddpcie950.obj
 0001:00000628       ??_7CPddpcie950@@6BCMiniThread@@@ 10001628     pddpcie950:pddpcie950.obj
 0001:00000630       ??_7CPddpcie950@@6BCSerialPDD@@@ 10001630     pddpcie950:pddpcie950.obj
 0001:00000734       ??_7CPddpcie950Isr@@6BCMiniThread@@@ 10001734     pddpcie950:pddisrpcie950.obj
 0001:00000738       ??_7CPddpcie950Isr@@6BCSerialPDD@@@ 10001738     pddpcie950:pddisrpcie950.obj
 0001:0000083c       ??_C@_1BE@GPBAGNPC@?$AAI?$AAs?$AAr?$AAH?$AAa?$AAn?$AAd?$AAl?$AAe?$AA?$AA@ 1000183c     pddpcie950:pddisrpcie950.obj
 0001:00000850       ??_C@_1CA@INOAHGHF@?$AAB?$AAu?$AAs?$AAA?$AAc?$AAc?$AAe?$AAs?$AAs?$AAH?$AAa?$AAn?$AAd?$AAl?$AAe?$AA?$AA@ 10001850     pddpcie950:pddisrpcie950.obj
 0001:00000870       ??_C@_1BC@MCDIKBIL@?$AAI?$AAs?$AAt?$AAE?$AAv?$AAe?$AAn?$AAt?$AA?$AA@ 10001870     pddpcie950:pddisrpcie950.obj
 0001:00000884       ??_C@_1BG@LJAMCNJN@?$AAP?$AAo?$AAr?$AAt?$AAN?$AAu?$AAm?$AAb?$AAe?$AAr?$AA?$AA@ 10001884     pddpcie950:pddisrpcie950.obj
 0001:000008a0       ??_C@_1GC@BNHHHKJC@?$AAp?$AAd?$AAd?$AAi?$AAs?$AAr?$AAp?$AAc?$AAi?$AAe?$AA9?$AA5?$AA0?$AA?3?$AA?5?$AAC?$AAo?$AAd?$AAe?$AA?5?$AA?$DN?$AA?5?$AAE?$AAX?$AAC?$AAE?$AAP?$AAT?$AAI?$AAO?$AAN?$AA_@ 100018a0     pddpcie950:pddisrpcie950.obj
 0001:00000908       ??_C@_1EI@KIOAGNNB@?$AAp?$AAd?$AAd?$AAi?$AAs?$AAr?$AAp?$AAc?$AAi?$AAe?$AA9?$AA5?$AA0?$AA?3?$AA?5?$AAI?$AAn?$AA?5?$AAf?$AAi?$AAl?$AAt?$AAe?$AAr?$AA?4?$AA?5?$AAC?$AAo?$AAd?$AAe?$AA?5?$AA?$DN@ 10001908     pddpcie950:pddisrpcie950.obj
 0001:00000950       ??_C@_1DC@LJHLBINO@?$AAp?$AAd?$AAd?$AAi?$AAs?$AAr?$AAp?$AAc?$AAi?$AAe?$AA9?$AA5?$AA0?$AA?3?$AA?5?$AAI?$AAn?$AA?5?$AAE?$AAx?$AAc?$AAe?$AAp?$AAt?$AA?$AA@ 10001950     pddpcie950:pddisrpcie950.obj
 0001:00000988       __load_config_used         10001988     corelib0:loadcfg.obj
 0001:00000a00       ___safe_se_handler_table   10001a00     <linker-defined>
 0001:00000a04       ?CreateSerialObject@@YAPAVCSerialPDD@@PAGPAXPAU__HWOBJ@@K@Z 10001a04 f   compcie950.obj
 0001:00000a93       ?DeleteSerialObject@@YAXPAVCSerialPDD@@@Z 10001a93 f   compcie950.obj
 0001:00000aa5       ?RxBytesAvail@@YAKPAU__HW_INDEP_INFO@@@Z 10001aa5 f i mddpcie950:mddpcie950.obj
 0001:00000acd       ?DoTxData@@YAXPAU__HW_INDEP_INFO@@@Z 10001acd f   mddpcie950:mddpcie950.obj
 0001:00000bf6       ?DoRxData@@YAKPAU__HW_INDEP_INFO@@@Z 10001bf6 f   mddpcie950:mddpcie950.obj
 0001:00000c8b       ?StopDispatchThread@@YAHPAU__HW_INDEP_INFO@@@Z 10001c8b f   mddpcie950:mddpcie950.obj
 0001:00000d03       ?ApplyDCB@@YAHPAU__HW_INDEP_INFO@@PAU_DCB@@H@Z 10001d03 f   mddpcie950:mddpcie950.obj
 0001:00000d50       ?COM_PreClose@@YAXPAU__HW_OPEN_INFO@@@Z 10001d50 f   mddpcie950:mddpcie950.obj
 0001:00000df3       ?COM_Close@@YAHPAU__HW_OPEN_INFO@@@Z 10001df3 f   mddpcie950:mddpcie950.obj
 0001:00000ef1       ?ProcessExiting@@YAHPAU__HW_OPEN_INFO@@@Z 10001ef1 f   mddpcie950:mddpcie950.obj
 0001:00000f14       ?COM_PreDeinit@@YAHPAU__HW_INDEP_INFO@@@Z 10001f14 f   mddpcie950:mddpcie950.obj
 0001:00000f6c       ?COM_Deinit@@YAHPAU__HW_INDEP_INFO@@@Z 10001f6c f   mddpcie950:mddpcie950.obj
 0001:00001070       ?COM_Read@@YAKPAXPAEK@Z    10002070 f   mddpcie950:mddpcie950.obj
 0001:0000128a       ?COM_Seek@@YAKPAXJK@Z      1000228a f   mddpcie950:mddpcie950.obj
 0001:0000128e       ?COM_PowerUp@@YAHPAX@Z     1000228e f   mddpcie950:mddpcie950.obj
 0001:000012af       ?COM_PowerDown@@YAHPAX@Z   100022af f   mddpcie950:mddpcie950.obj
 0001:000012d0       ?WaitCommEvent@@YAHPAU__HW_OPEN_INFO@@PAKPAU_OVERLAPPED@@@Z 100022d0 f   mddpcie950:mddpcie950.obj
 0001:000013ab       _EvaluateEventFlag         100023ab f   mddpcie950:mddpcie950.obj
 0001:0000142c       ?COM_IOControl@@YAHPAU__HW_OPEN_INFO@@KPAEK1KPAK@Z 1000242c f   mddpcie950:mddpcie950.obj
 0001:00001b71       _SerialEventHandler        10002b71 f   mddpcie950:mddpcie950.obj
 0001:00001c97       ?StartDispatchThread@@YAHPAU__HW_INDEP_INFO@@@Z 10002c97 f   mddpcie950:mddpcie950.obj
 0001:00001cef       ?COM_Init@@YAPAXK@Z        10002cef f   mddpcie950:mddpcie950.obj
 0001:00001f09       ?COM_Open@@YAPAXPAXKK@Z    10002f09 f   mddpcie950:mddpcie950.obj
 0001:0000213a       ?COM_Write@@YAKPAXPAEK@Z   1000313a f   mddpcie950:mddpcie950.obj
 0001:000022d5       ??0CRegistryEdit@@QAE@PBG@Z 100032d5 f i serpcie950:serpcie950.obj
 0001:000022f6       ?GetRegValue@CRegistryEdit@@QAEHPBGPAEK@Z 100032f6 f i serpcie950:serpcie950.obj
 0001:00002322       ?ThreadStart@CMiniThread@@QAEHXZ 10003322 f i serpcie950:serpcie950.obj
 0001:00002347       ?WaitThreadComplete@CMiniThread@@QAEHK@Z 10003347 f i serpcie950:serpcie950.obj
 0001:00002388       ?ForceTerminated@CMiniThread@@QAEHXZ 10003388 f i serpcie950:serpcie950.obj
 0001:000023bb       ?ThreadProc@CMiniThread@@CAKPAX@Z 100033bb f i serpcie950:serpcie950.obj
 0001:000023d8       ?SignalCallback@CSerialPDDPowerUpCallback@@QAEHXZ 100033d8 f i serpcie950:serpcie950.obj
 0001:000023ed       ?SignalCallback@CSerialPDDPowerUpCallback@@QAEHK@Z 100033ed f i serpcie950:serpcie950.obj
 0001:00002404       ?ThreadRun@CSerialPDDPowerUpCallback@@EAEKXZ 10003404 f   serpcie950:serpcie950.obj
 0001:0000243f       ??0CSerialPDD@@QAE@PAGPAXPAU__HWOBJ@@@Z 1000343f f   serpcie950:serpcie950.obj
 0001:0000250f       ?GetDevicePowerState@CSerialPDD@@UAE?AW4_CEDEVICE_POWER_STATE@@XZ 1000350f f i serpcie950:serpcie950.obj
 0001:00002513       ?GetPowerCapabilities@CSerialPDD@@UAE?AU_POWER_CAPABILITIES@@XZ 10003513 f i serpcie950:serpcie950.obj
 0001:0000252b       ?IsCTSOff@CSerialPDD@@UAEHXZ 1000352b f i serpcie950:serpcie950.obj
 0001:0000253c       ?IsDSROff@CSerialPDD@@UAEHXZ 1000353c f i serpcie950:serpcie950.obj
 0001:0000254d       ?SetInternalLoopback@CSerialPDD@@UAEXH@Z 1000354d f i serpcie950:serpcie950.obj
 0001:00002550       ?RegSetPnpValue@CSerialPDD@@UAEHPBGKPBEK@Z 10003550 f i serpcie950:serpcie950.obj
 0001:00002555       ?SetLineDriverControls@CSerialPDD@@UAEHPAULINE_DRIVER_CONTROL@@K@Z 10003555 f i serpcie950:serpcie950.obj
 0001:00002555       ?GetLineDriverControls@CSerialPDD@@UAEHPAULINE_DRIVER_CONTROL@@K@Z 10003555 f i serpcie950:serpcie950.obj
 0001:0000255a       ?SaveBaudrateMap@CSerialPDD@@UAEHPAUBAUDRATE_MAP@@@Z 1000355a f i serpcie950:serpcie950.obj
 0001:0000255a       ?SaveLineDriverControls@CSerialPDD@@UAEHPAULINE_DRIVER_CONTROL@@@Z 1000355a f i serpcie950:serpcie950.obj
 0001:0000255a       ?SetFifoCtrlLevels@CSerialPDD@@UAEHPAUFIFO_LEVEL_CTRL_VALS@@@Z 1000355a f i serpcie950:serpcie950.obj
 0001:0000255f       ?SetOutputMode@CSerialPDD@@UAEXHH@Z 1000355f f i serpcie950:serpcie950.obj
 0001:00002578       ?GetOutputMode@CSerialPDD@@UAEXPAH0@Z 10003578 f i serpcie950:serpcie950.obj
 0001:0000259d       ?PostInit@CSerialPDD@@UAEXXZ 1000359d f   serpcie950:serpcie950.obj
 0001:000025b2       ?Open@CSerialPDD@@UAEHXZ   100035b2 f   serpcie950:serpcie950.obj
 0001:00002601       ?Close@CSerialPDD@@UAEHXZ  10003601 f   serpcie950:serpcie950.obj
 0001:0000264f       ?Reset@CSerialPDD@@QAEXXZ  1000364f f   serpcie950:serpcie950.obj
 0001:0000268a       ?Ioctl@CSerialPDD@@UAEHKPAEK0KPAK@Z 1000368a f   serpcie950:serpcie950.obj
 0001:00002918       ?InitialPower@CSerialPDD@@UAEHH@Z 10003918 f   serpcie950:serpcie950.obj
 0001:00002926       ?SetPowerStateStatic@CSerialPDD@@KA?AW4_CEDEVICE_POWER_STATE@@KW42@@Z 10003926 f   serpcie950:serpcie950.obj
 0001:00002948       ?PowerOff@CSerialPDD@@UAEHXZ 10003948 f   serpcie950:serpcie950.obj
 0001:0000296f       ?PowerOn@CSerialPDD@@UAEHXZ 1000396f f   serpcie950:serpcie950.obj
 0001:000029ba       ?SetDevicePowerState@CSerialPDD@@UAEHW4_CEDEVICE_POWER_STATE@@@Z 100039ba f   serpcie950:serpcie950.obj
 0001:00002a34       ?InitialEnableInterrupt@CSerialPDD@@UAEHH@Z 10003a34 f   serpcie950:serpcie950.obj
 0001:00002a55       ?NotifyPDDInterrupt@CSerialPDD@@UAEHW4INTERRUPT_TYPE@@@Z 10003a55 f   serpcie950:serpcie950.obj
 0001:00002aba       ?GetInterruptType@CSerialPDD@@UAE?AW4INTERRUPT_TYPE@@XZ 10003aba f   serpcie950:serpcie950.obj
 0001:00002add       ?DataReplaced@CSerialPDD@@UAEHPAEH@Z 10003add f   serpcie950:serpcie950.obj
 0001:00002b5c       ?EventCallback@CSerialPDD@@UAEHKK@Z 10003b5c f   serpcie950:serpcie950.obj
 0001:00002b94       ?PurgeComm@CSerialPDD@@UAEHK@Z 10003b94 f   serpcie950:serpcie950.obj
 0001:00002bba       ?SetReceiveError@CSerialPDD@@UAEXK@Z 10003bba f   serpcie950:serpcie950.obj
 0001:00002bf5       ?GetReceivedError@CSerialPDD@@UAEKXZ 10003bf5 f   serpcie950:serpcie950.obj
 0001:00002c1a       ?SetDefaultConfiguration@CSerialPDD@@UAEXXZ 10003c1a f   serpcie950:serpcie950.obj
 0001:00002cf5       ?SetDCB@CSerialPDD@@UAEHPAU_DCB@@@Z 10003cf5 f   serpcie950:serpcie950.obj
 0001:00002e39       ?SerInit@@YAPAXKPAXPAU__HWOBJ@@@Z 10003e39 f   serpcie950:serpcie950.obj
 0001:00002e70       ?SerDeinit@@YAKPAX@Z       10003e70 f   serpcie950:serpcie950.obj
 0001:00002e9a       ?SerPostInit@@YAHPAX@Z     10003e9a f   serpcie950:serpcie950.obj
 0001:00002eae       ?SerOpen@@YAHPAX@Z         10003eae f   serpcie950:serpcie950.obj
 0001:00002ec2       ?SerClose@@YAKPAX@Z        10003ec2 f   serpcie950:serpcie950.obj
 0001:00002ed6       ?SerGetInterruptType@@YA?AW4INTERRUPT_TYPE@@PAX@Z 10003ed6 f   serpcie950:serpcie950.obj
 0001:00002eea       ?SerRxIntr@@YAKPAXPAEPAK@Z 10003eea f   serpcie950:serpcie950.obj
 0001:00002f03       ?SerTxIntrEx@@YAXPAXPAEPAK@Z 10003f03 f   serpcie950:serpcie950.obj
 0001:00002f1a       ?SerModemIntr@@YAXPAX@Z    10003f1a f   serpcie950:serpcie950.obj
 0001:00002f2c       ?SerLineIntr@@YAXPAX@Z     10003f2c f   serpcie950:serpcie950.obj
 0001:00002f41       ?SerGetRxBufferSize@@YAKPAX@Z 10003f41 f   serpcie950:serpcie950.obj
 0001:00002f58       ?SerPowerOff@@YAHPAX@Z     10003f58 f   serpcie950:serpcie950.obj
 0001:00002f6c       ?SerPowerOn@@YAHPAX@Z      10003f6c f   serpcie950:serpcie950.obj
 0001:00002f80       ?SerClearDTR@@YAXPAX@Z     10003f80 f   serpcie950:serpcie950.obj
 0001:00002f96       ?SerSetDTR@@YAXPAX@Z       10003f96 f   serpcie950:serpcie950.obj
 0001:00002fac       ?SerClearRTS@@YAXPAX@Z     10003fac f   serpcie950:serpcie950.obj
 0001:00002fc2       ?SerSetRTS@@YAXPAX@Z       10003fc2 f   serpcie950:serpcie950.obj
 0001:00002fd8       ?SerEnableIR@@YAHPAXK@Z    10003fd8 f   serpcie950:serpcie950.obj
 0001:00003006       ?SerDisableIR@@YAHPAX@Z    10004006 f   serpcie950:serpcie950.obj
 0001:00003021       ?SerClearBreak@@YAXPAX@Z   10004021 f   serpcie950:serpcie950.obj
 0001:00003037       ?SerSetBreak@@YAXPAX@Z     10004037 f   serpcie950:serpcie950.obj
 0001:0000304d       ?SerXmitComChar@@YAHPAXE@Z 1000404d f   serpcie950:serpcie950.obj
 0001:00003064       ?SerGetStatus@@YAKPAXPAU_COMSTAT@@@Z 10004064 f   serpcie950:serpcie950.obj
 0001:00003113       ?SerReset@@YAXPAX@Z        10004113 f   serpcie950:serpcie950.obj
 0001:00003125       ?SerGetModemStatus@@YAXPAXPAK@Z 10004125 f   serpcie950:serpcie950.obj
 0001:00003144       ?SerGetCommProperties@@YAXPAXPAU_COMMPROP@@@Z 10004144 f   serpcie950:serpcie950.obj
 0001:00003166       ?SerPurgeComm@@YAXPAXK@Z   10004166 f   serpcie950:serpcie950.obj
 0001:0000317a       ?SerSetDCB@@YAHPAXPAU_DCB@@@Z 1000417a f   serpcie950:serpcie950.obj
 0001:00003198       ?SerSetCommTimeouts@@YAHPAXPAU_COMMTIMEOUTS@@@Z 10004198 f   serpcie950:serpcie950.obj
 0001:0000319c       ?SerEnableXmit@@YAXPAXH@Z  1000419c f   serpcie950:serpcie950.obj
 0001:000031b3       ?SerIoctl@@YAHPAXKPAEK1KPAK@Z 100041b3 f   serpcie950:serpcie950.obj
 0001:000031d8       _GetSerialObject           100041d8 f   serpcie950:serpcie950.obj
 0001:000031fe       ??0CMiniThread@@QAE@KH@Z   100041fe f i serpcie950:serpcie950.obj
 0001:00003245       ??0CSerialPDDPowerUpCallback@@QAE@PAVCSerialPDD@@@Z 10004245 f   serpcie950:serpcie950.obj
 0001:00003281       ??1CSerialPDDPowerUpCallback@@QAE@XZ 10004281 f   serpcie950:serpcie950.obj
 0001:000032b4       ??_GCSerialPDDPowerUpCallback@@QAEPAXI@Z 100042b4 f i serpcie950:serpcie950.obj
 0001:000032d3       ?Init@CSerialPDD@@UAEHXZ   100042d3 f   serpcie950:serpcie950.obj
 0001:00003340       ??1CSerialPDD@@UAE@XZ      10004340 f   serpcie950:serpcie950.obj
 0001:000033a8       ??_GCSerialPDD@@UAEPAXI@Z  100043a8 f i serpcie950:serpcie950.obj
 0001:000033a8       ??_ECSerialPDD@@UAEPAXI@Z  100043a8 f i serpcie950:serpcie950.obj
 0001:000033c7       ??0CRegistryEdit@@QAE@PAUHKEY__@@PBG@Z 100043c7 f i pddpcie950:pddpcie950.obj
 0001:000033f7       ?GetWindowInfo@CRegistryEdit@@QAEKPAU_DDKWINDOWINFO_tag@@@Z 100043f7 f i pddpcie950:pddpcie950.obj
 0001:0000341f       ?RegQueryValueExW@CRegistryEdit@@QAEHPBGPAKPAE1@Z 1000441f f i pddpcie950:pddpcie950.obj
 0001:00003444       ?CeSetPriority@CMiniThread@@QAEHH@Z 10004444 f i pddpcie950:pddpcie950.obj
 0001:00003462       ??1CRegpcie950@@UAE@XZ     10004462 f i pddpcie950:pddpcie950.obj
 0001:00003476       ?Init@CRegpcie950@@UAEHXZ  10004476 f i pddpcie950:pddpcie950.obj
 0001:0000347f       ?Write_DATA@CRegpcie950@@UAEXE@Z 1000447f f i pddpcie950:pddpcie950.obj
 0001:00003493       ?Read_Data@CRegpcie950@@UAEEXZ 10004493 f i pddpcie950:pddpcie950.obj
 0001:0000349d       ?Write_IER@CRegpcie950@@UAEXE@Z 1000449d f i pddpcie950:pddpcie950.obj
 0001:000034b1       ?Read_IER@CRegpcie950@@UAEEXZ 100044b1 f i pddpcie950:pddpcie950.obj
 0001:000034bb       ?Write_FCR@CRegpcie950@@UAEXE@Z 100044bb f i pddpcie950:pddpcie950.obj
 0001:000034dc       ?Read_FCR@CRegpcie950@@UAEEXZ 100044dc f i pddpcie950:pddpcie950.obj
 0001:000034e0       ?Read_IIR@CRegpcie950@@UAEEXZ 100044e0 f i pddpcie950:pddpcie950.obj
 0001:000034ea       ?Write_LCR@CRegpcie950@@UAEXE@Z 100044ea f i pddpcie950:pddpcie950.obj
 0001:000034fe       ?Read_LCR@CRegpcie950@@UAEEXZ 100044fe f i pddpcie950:pddpcie950.obj
 0001:00003508       ?Write_MCR@CRegpcie950@@UAEXE@Z 10004508 f i pddpcie950:pddpcie950.obj
 0001:0000351c       ?Read_MCR@CRegpcie950@@UAEEXZ 1000451c f i pddpcie950:pddpcie950.obj
 0001:00003526       ?Write_LSR@CRegpcie950@@UAEXE@Z 10004526 f i pddpcie950:pddpcie950.obj
 0001:0000353a       ?Read_LSR@CRegpcie950@@UAEEXZ 1000453a f i pddpcie950:pddpcie950.obj
 0001:00003544       ?Write_MSR@CRegpcie950@@UAEXE@Z 10004544 f i pddpcie950:pddpcie950.obj
 0001:00003558       ?Read_MSR@CRegpcie950@@UAEEXZ 10004558 f i pddpcie950:pddpcie950.obj
 0001:00003562       ?Write_SPR@CRegpcie950@@UAEXE@Z 10004562 f i pddpcie950:pddpcie950.obj
 0001:00003576       ?Read_SPR@CRegpcie950@@UAEEXZ 10004576 f i pddpcie950:pddpcie950.obj
 0001:00003580       ?Write_DIVISOR@CRegpcie950@@UAEXG@Z 10004580 f i pddpcie950:pddpcie950.obj
 0001:000035a9       ?Read_DIVISOR@CRegpcie950@@UAEGXZ 100045a9 f i pddpcie950:pddpcie950.obj
 0001:000035d6       ?Write_EFR@CRegpcie950@@UAEXE@Z 100045d6 f i pddpcie950:pddpcie950.obj
 0001:000035eb       ?Read_EFR@CRegpcie950@@UAEEXZ 100045eb f i pddpcie950:pddpcie950.obj
 0001:000035f7       ?Write_XON1@CRegpcie950@@UAEXE@Z 100045f7 f i pddpcie950:pddpcie950.obj
 0001:0000360c       ?Read_XON1@CRegpcie950@@UAEEXZ 1000460c f i pddpcie950:pddpcie950.obj
 0001:00003618       ?Write_XON2@CRegpcie950@@UAEXE@Z 10004618 f i pddpcie950:pddpcie950.obj
 0001:0000362d       ?Read_XON2@CRegpcie950@@UAEEXZ 1000462d f i pddpcie950:pddpcie950.obj
 0001:00003639       ?Write_XOFF1@CRegpcie950@@UAEXE@Z 10004639 f i pddpcie950:pddpcie950.obj
 0001:0000364e       ?Read_XOFF1@CRegpcie950@@UAEEXZ 1000464e f i pddpcie950:pddpcie950.obj
 0001:0000365a       ?Write_XOFF2@CRegpcie950@@UAEXE@Z 1000465a f i pddpcie950:pddpcie950.obj
 0001:0000366f       ?Read_XOFF2@CRegpcie950@@UAEEXZ 1000466f f i pddpcie950:pddpcie950.obj
 0001:0000367b       ?Write_ASR@CRegpcie950@@UAEXE@Z 1000467b f i pddpcie950:pddpcie950.obj
 0001:00003690       ?Read_ASR@CRegpcie950@@UAEEXZ 10004690 f i pddpcie950:pddpcie950.obj
 0001:0000369c       ?Read_RFL@CRegpcie950@@UAEEXZ 1000469c f i pddpcie950:pddpcie950.obj
 0001:000036c3       ?Read_TFL@CRegpcie950@@UAEEXZ 100046c3 f i pddpcie950:pddpcie950.obj
 0001:000036ea       ?Write_ACR@CRegpcie950@@UAEXE@Z 100046ea f i pddpcie950:pddpcie950.obj
 0001:000036ff       ?Read_ACR@CRegpcie950@@UAEEXZ 100046ff f i pddpcie950:pddpcie950.obj
 0001:0000370b       ?Write_CPR@CRegpcie950@@UAEXE@Z 1000470b f i pddpcie950:pddpcie950.obj
 0001:00003720       ?Read_CPR@CRegpcie950@@UAEEXZ 10004720 f i pddpcie950:pddpcie950.obj
 0001:0000372c       ?Write_TCR@CRegpcie950@@UAEXE@Z 1000472c f i pddpcie950:pddpcie950.obj
 0001:00003741       ?Read_TCR@CRegpcie950@@UAEEXZ 10004741 f i pddpcie950:pddpcie950.obj
 0001:0000374d       ?Write_TTL@CRegpcie950@@UAEXE@Z 1000474d f i pddpcie950:pddpcie950.obj
 0001:00003762       ?Read_TTL@CRegpcie950@@UAEEXZ 10004762 f i pddpcie950:pddpcie950.obj
 0001:0000376e       ?Write_RTL@CRegpcie950@@UAEXE@Z 1000476e f i pddpcie950:pddpcie950.obj
 0001:00003783       ?Read_RTL@CRegpcie950@@UAEEXZ 10004783 f i pddpcie950:pddpcie950.obj
 0001:0000378f       ?Write_FCL@CRegpcie950@@UAEXE@Z 1000478f f i pddpcie950:pddpcie950.obj
 0001:000037a4       ?Read_FCL@CRegpcie950@@UAEEXZ 100047a4 f i pddpcie950:pddpcie950.obj
 0001:000037b0       ?Write_FCH@CRegpcie950@@UAEXE@Z 100047b0 f i pddpcie950:pddpcie950.obj
 0001:000037c8       ?Read_FCH@CRegpcie950@@UAEEXZ 100047c8 f i pddpcie950:pddpcie950.obj
 0001:000037d7       ?Write_NMR@CRegpcie950@@UAEXE@Z 100047d7 f i pddpcie950:pddpcie950.obj
 0001:000037ef       ?Read_NMR@CRegpcie950@@UAEEXZ 100047ef f i pddpcie950:pddpcie950.obj
 0001:000037fe       ?Write_MDM@CRegpcie950@@UAEXE@Z 100047fe f i pddpcie950:pddpcie950.obj
 0001:00003816       ?Read_MDM@CRegpcie950@@UAEEXZ 10004816 f i pddpcie950:pddpcie950.obj
 0001:00003825       ?Write_485CR@CRegpcie950@@UAEXE@Z 10004825 f i pddpcie950:pddpcie950.obj
 0001:0000383d       ?Read_485CR@CRegpcie950@@UAEEXZ 1000483d f i pddpcie950:pddpcie950.obj
 0001:0000384c       ?Write_485DR@CRegpcie950@@UAEXE@Z 1000484c f i pddpcie950:pddpcie950.obj
 0001:00003864       ?Read_485DR@CRegpcie950@@UAEEXZ 10004864 f i pddpcie950:pddpcie950.obj
 0001:00003873       ?Read_ID1@CRegpcie950@@UAEEXZ 10004873 f i pddpcie950:pddpcie950.obj
 0001:00003882       ?Read_ID2@CRegpcie950@@UAEEXZ 10004882 f i pddpcie950:pddpcie950.obj
 0001:00003891       ?Read_ID3@CRegpcie950@@UAEEXZ 10004891 f i pddpcie950:pddpcie950.obj
 0001:000038a0       ?WRITE_550_PORT@CRegpcie950@@UAEXPAEE@Z 100048a0 f i pddpcie950:pddpcie950.obj
 0001:000038de       ?READ_550_PORT@CRegpcie950@@UAEEPAE@Z 100048de f i pddpcie950:pddpcie950.obj
 0001:0000391f       ?WRITE_ICR_PORT@CRegpcie950@@UAEXPAEE@Z 1000491f f i pddpcie950:pddpcie950.obj
 0001:0000391f       ?WRITE_650_PORT@CRegpcie950@@UAEXPAEE@Z 1000491f f i pddpcie950:pddpcie950.obj
 0001:0000391f       ?WRITE_950_PORT@CRegpcie950@@UAEXPAEE@Z 1000491f f i pddpcie950:pddpcie950.obj
 0001:00003933       ?READ_950_PORT@CRegpcie950@@UAEEPAE@Z 10004933 f i pddpcie950:pddpcie950.obj
 0001:00003933       ?READ_ICR_PORT@CRegpcie950@@UAEEPAE@Z 10004933 f i pddpcie950:pddpcie950.obj
 0001:00003933       ?READ_650_PORT@CRegpcie950@@UAEEPAE@Z 10004933 f i pddpcie950:pddpcie950.obj
 0001:00003943       ??0CRegpcie950@@QAE@PAEK@Z 10004943 f   pddpcie950:pddpcie950.obj
 0001:00003b11       ?Backup@CRegpcie950@@UAEXXZ 10004b11 f   pddpcie950:pddpcie950.obj
 0001:00003c4e       ?Restore@CRegpcie950@@UAEXXZ 10004c4e f   pddpcie950:pddpcie950.obj
 0001:00003da2       ?Init@CPddpcie950@@UAEHXZ  10004da2 f   pddpcie950:pddpcie950.obj
 0001:00003fe8       ?GetRegMultiDword@CPddpcie950@@EAEHPBGPAKK@Z 10004fe8 f   pddpcie950:pddpcie950.obj
 0001:00004089       ?MapHardware@CPddpcie950@@UAEHXZ 10005089 f   pddpcie950:pddpcie950.obj
 0001:000041b6       ?PostInit@CPddpcie950@@UAEXXZ 100051b6 f   pddpcie950:pddpcie950.obj
 0001:0000428d       ?ThreadRun@CPddpcie950@@EAEKXZ 1000528d f   pddpcie950:pddpcie950.obj
 0001:00004378       ?InitialEnableInterrupt@CPddpcie950@@UAEHH@Z 10005378 f   pddpcie950:pddpcie950.obj
 0001:0000442a       ?InitXmit@CPddpcie950@@UAEHH@Z 1000542a f   pddpcie950:pddpcie950.obj
 0001:00004484       ?GetWriteableSize@CPddpcie950@@UAEKXZ 10005484 f   pddpcie950:pddpcie950.obj
 0001:0000449d       ?PushPriorityFifo@CPddpcie950@@IAEXE@Z 1000549d f   pddpcie950:pddpcie950.obj
 0001:00004520       ?PopPriorityFifo@CPddpcie950@@IAEHPAE@Z 10005520 f   pddpcie950:pddpcie950.obj
 0001:00004574       ?XmitComChar@CPddpcie950@@UAEXE@Z 10005574 f   pddpcie950:pddpcie950.obj
 0001:000045c1       ?EnableReceiveInterrupt@CPddpcie950@@UAEHH@Z 100055c1 f   pddpcie950:pddpcie950.obj
 0001:0000462d       ?EnableXmitInterrupt@CPddpcie950@@UAEHH@Z 1000562d f   pddpcie950:pddpcie950.obj
 0001:00004699       ?CancelXmit@CPddpcie950@@UAEHXZ 10005699 f   pddpcie950:pddpcie950.obj
 0001:000046cf       ?EmptyEventData@CPddpcie950@@UAEXXZ 100056cf f   pddpcie950:pddpcie950.obj
 0001:000046d0       ?InitReceive@CPddpcie950@@UAEHH@Z 100056d0 f   pddpcie950:pddpcie950.obj
 0001:00004758       ?GetReadableSize@CPddpcie950@@IAEKXZ 10005758 f   pddpcie950:pddpcie950.obj
 0001:00004783       ?ReceiveInterruptHandler@CPddpcie950@@UAEKPAEPAK@Z 10005783 f   pddpcie950:pddpcie950.obj
 0001:0000482d       ?CancelReceive@CPddpcie950@@UAEKXZ 1000582d f   pddpcie950:pddpcie950.obj
 0001:00004869       ?InitModem@CPddpcie950@@UAEHH@Z 10005869 f   pddpcie950:pddpcie950.obj
 0001:000048cd       ?GetModemStatus@CPddpcie950@@UAEKXZ 100058cd f   pddpcie950:pddpcie950.obj
 0001:00004932       ?SetDTR@CPddpcie950@@UAEXH@Z 10005932 f   pddpcie950:pddpcie950.obj
 0001:0000497d       ?SetRTS@CPddpcie950@@UAEXH@Z 1000597d f   pddpcie950:pddpcie950.obj
 0001:000049c8       ?InitLine@CPddpcie950@@UAEHH@Z 100059c8 f   pddpcie950:pddpcie950.obj
 0001:00004a36       ?GetLineStatus@CPddpcie950@@QAEEXZ 10005a36 f   pddpcie950:pddpcie950.obj
 0001:00004a85       ?SetBreak@CPddpcie950@@UAEXH@Z 10005a85 f   pddpcie950:pddpcie950.obj
 0001:00004ad0       ?GetBaudConfigFromBaudRate@CPddpcie950@@IAEHKJPAU_BAUD_CONFIG@1@@Z 10005ad0 f   pddpcie950:pddpcie950.obj
 0001:00004bca       ?SetBaudRate@CPddpcie950@@UAEHKH@Z 10005bca f   pddpcie950:pddpcie950.obj
 0001:00004c6e       ?SetByteSize@CPddpcie950@@UAEHK@Z 10005c6e f   pddpcie950:pddpcie950.obj
 0001:00004cd4       ?SetParity@CPddpcie950@@UAEHK@Z 10005cd4 f   pddpcie950:pddpcie950.obj
 0001:00004d33       ?SetStopBits@CPddpcie950@@UAEHK@Z 10005d33 f   pddpcie950:pddpcie950.obj
 0001:00004d7b       ?SetFlowControl@CPddpcie950@@UAEHPAU_DCB@@@Z 10005d7b f   pddpcie950:pddpcie950.obj
 0001:00004f46       ?GetXonXoffStatus@CPddpcie950@@UAEXPAU_COMSTAT@@@Z 10005f46 f   pddpcie950:pddpcie950.obj
 0001:00004f97       ?EnableXmit@CPddpcie950@@UAEXH@Z 10005f97 f   pddpcie950:pddpcie950.obj
 0001:00004fd5       ?SetFifoCtrlLevels@CPddpcie950@@UAEHPAUFIFO_LEVEL_CTRL_VALS@@@Z 10005fd5 f   pddpcie950:pddpcie950.obj
 0001:00005127       ?SetInternalLoopback@CPddpcie950@@UAEXH@Z 10006127 f   pddpcie950:pddpcie950.obj
 0001:00005157       ?GetLineDriverControls@CPddpcie950@@UAEHPAULINE_DRIVER_CONTROL@@K@Z 10006157 f   pddpcie950:pddpcie950.obj
 0001:000051dd       ?SetLineDriverControls@CPddpcie950@@UAEHPAULINE_DRIVER_CONTROL@@K@Z 100061dd f   pddpcie950:pddpcie950.obj
 0001:00005299       ?SaveLineDriverControls@CPddpcie950@@UAEHPAULINE_DRIVER_CONTROL@@@Z 10006299 f   pddpcie950:pddpcie950.obj
 0001:000052fb       ?SaveBaudrateMap@CPddpcie950@@UAEHPAUBAUDRATE_MAP@@@Z 100062fb f   pddpcie950:pddpcie950.obj
 0001:00005535       ?RegSetPnpValue@CPddpcie950@@UAEHPBGKPBEK@Z 10006535 f   pddpcie950:pddpcie950.obj
 0001:000056db       ??0CMemRegpcie950@@QAE@PAEK@Z 100066db f i pddpcie950:pddpcie950.obj
 0001:000056f9       ?Write_DATA@CMemRegpcie950@@UAEXE@Z 100066f9 f i pddpcie950:pddpcie950.obj
 0001:0000570d       ?Read_Data@CMemRegpcie950@@UAEEXZ 1000670d f i pddpcie950:pddpcie950.obj
 0001:00005717       ?Write_IER@CMemRegpcie950@@UAEXE@Z 10006717 f i pddpcie950:pddpcie950.obj
 0001:0000572b       ?Read_IER@CMemRegpcie950@@UAEEXZ 1000672b f i pddpcie950:pddpcie950.obj
 0001:00005735       ?Write_FCR@CMemRegpcie950@@UAEXE@Z 10006735 f i pddpcie950:pddpcie950.obj
 0001:00005756       ?Read_IIR@CMemRegpcie950@@UAEEXZ 10006756 f i pddpcie950:pddpcie950.obj
 0001:00005760       ?Write_LCR@CMemRegpcie950@@UAEXE@Z 10006760 f i pddpcie950:pddpcie950.obj
 0001:00005774       ?Read_LCR@CMemRegpcie950@@UAEEXZ 10006774 f i pddpcie950:pddpcie950.obj
 0001:0000577e       ?Write_MCR@CMemRegpcie950@@UAEXE@Z 1000677e f i pddpcie950:pddpcie950.obj
 0001:00005792       ?Read_MCR@CMemRegpcie950@@UAEEXZ 10006792 f i pddpcie950:pddpcie950.obj
 0001:0000579c       ?Write_LSR@CMemRegpcie950@@UAEXE@Z 1000679c f i pddpcie950:pddpcie950.obj
 0001:000057b0       ?Read_LSR@CMemRegpcie950@@UAEEXZ 100067b0 f i pddpcie950:pddpcie950.obj
 0001:000057ba       ?Write_MSR@CMemRegpcie950@@UAEXE@Z 100067ba f i pddpcie950:pddpcie950.obj
 0001:000057ce       ?Read_MSR@CMemRegpcie950@@UAEEXZ 100067ce f i pddpcie950:pddpcie950.obj
 0001:000057d8       ?Write_SPR@CMemRegpcie950@@UAEXE@Z 100067d8 f i pddpcie950:pddpcie950.obj
 0001:000057ec       ?Read_SPR@CMemRegpcie950@@UAEEXZ 100067ec f i pddpcie950:pddpcie950.obj
 0001:000057f6       ?Write_DIVISOR@CMemRegpcie950@@UAEXG@Z 100067f6 f i pddpcie950:pddpcie950.obj
 0001:0000581f       ?Read_DIVISOR@CMemRegpcie950@@UAEGXZ 1000681f f i pddpcie950:pddpcie950.obj
 0001:0000584c       ?Write_EFR@CMemRegpcie950@@UAEXE@Z 1000684c f i pddpcie950:pddpcie950.obj
 0001:00005861       ?Read_EFR@CMemRegpcie950@@UAEEXZ 10006861 f i pddpcie950:pddpcie950.obj
 0001:0000586d       ?Write_XON1@CMemRegpcie950@@UAEXE@Z 1000686d f i pddpcie950:pddpcie950.obj
 0001:00005882       ?Read_XON1@CMemRegpcie950@@UAEEXZ 10006882 f i pddpcie950:pddpcie950.obj
 0001:0000588e       ?Write_XON2@CMemRegpcie950@@UAEXE@Z 1000688e f i pddpcie950:pddpcie950.obj
 0001:000058a3       ?Read_XON2@CMemRegpcie950@@UAEEXZ 100068a3 f i pddpcie950:pddpcie950.obj
 0001:000058af       ?Write_XOFF1@CMemRegpcie950@@UAEXE@Z 100068af f i pddpcie950:pddpcie950.obj
 0001:000058c4       ?Read_XOFF1@CMemRegpcie950@@UAEEXZ 100068c4 f i pddpcie950:pddpcie950.obj
 0001:000058d0       ?Write_XOFF2@CMemRegpcie950@@UAEXE@Z 100068d0 f i pddpcie950:pddpcie950.obj
 0001:000058e5       ?Read_XOFF2@CMemRegpcie950@@UAEEXZ 100068e5 f i pddpcie950:pddpcie950.obj
 0001:000058f1       ?Write_ASR@CMemRegpcie950@@UAEXE@Z 100068f1 f i pddpcie950:pddpcie950.obj
 0001:00005906       ?Read_ASR@CMemRegpcie950@@UAEEXZ 10006906 f i pddpcie950:pddpcie950.obj
 0001:00005912       ?Read_RFL@CMemRegpcie950@@UAEEXZ 10006912 f i pddpcie950:pddpcie950.obj
 0001:00005939       ?Read_TFL@CMemRegpcie950@@UAEEXZ 10006939 f i pddpcie950:pddpcie950.obj
 0001:00005960       ?Write_ACR@CMemRegpcie950@@UAEXE@Z 10006960 f i pddpcie950:pddpcie950.obj
 0001:00005975       ?Read_ACR@CMemRegpcie950@@UAEEXZ 10006975 f i pddpcie950:pddpcie950.obj
 0001:00005981       ?Write_CPR@CMemRegpcie950@@UAEXE@Z 10006981 f i pddpcie950:pddpcie950.obj
 0001:00005996       ?Read_CPR@CMemRegpcie950@@UAEEXZ 10006996 f i pddpcie950:pddpcie950.obj
 0001:000059a2       ?Write_TCR@CMemRegpcie950@@UAEXE@Z 100069a2 f i pddpcie950:pddpcie950.obj
 0001:000059b7       ?Read_TCR@CMemRegpcie950@@UAEEXZ 100069b7 f i pddpcie950:pddpcie950.obj
 0001:000059c3       ?Write_TTL@CMemRegpcie950@@UAEXE@Z 100069c3 f i pddpcie950:pddpcie950.obj
 0001:000059d8       ?Read_TTL@CMemRegpcie950@@UAEEXZ 100069d8 f i pddpcie950:pddpcie950.obj
 0001:000059e4       ?Write_RTL@CMemRegpcie950@@UAEXE@Z 100069e4 f i pddpcie950:pddpcie950.obj
 0001:000059f9       ?Read_RTL@CMemRegpcie950@@UAEEXZ 100069f9 f i pddpcie950:pddpcie950.obj
 0001:00005a05       ?Write_FCL@CMemRegpcie950@@UAEXE@Z 10006a05 f i pddpcie950:pddpcie950.obj
 0001:00005a1a       ?Read_FCL@CMemRegpcie950@@UAEEXZ 10006a1a f i pddpcie950:pddpcie950.obj
 0001:00005a26       ?Write_FCH@CMemRegpcie950@@UAEXE@Z 10006a26 f i pddpcie950:pddpcie950.obj
 0001:00005a3e       ?Read_FCH@CMemRegpcie950@@UAEEXZ 10006a3e f i pddpcie950:pddpcie950.obj
 0001:00005a4d       ?Write_NMR@CMemRegpcie950@@UAEXE@Z 10006a4d f i pddpcie950:pddpcie950.obj
 0001:00005a65       ?Read_NMR@CMemRegpcie950@@UAEEXZ 10006a65 f i pddpcie950:pddpcie950.obj
 0001:00005a74       ?Write_MDM@CMemRegpcie950@@UAEXE@Z 10006a74 f i pddpcie950:pddpcie950.obj
 0001:00005a8c       ?Read_MDM@CMemRegpcie950@@UAEEXZ 10006a8c f i pddpcie950:pddpcie950.obj
 0001:00005a9b       ?Write_485CR@CMemRegpcie950@@UAEXE@Z 10006a9b f i pddpcie950:pddpcie950.obj
 0001:00005ab3       ?Read_485CR@CMemRegpcie950@@UAEEXZ 10006ab3 f i pddpcie950:pddpcie950.obj
 0001:00005ac2       ?Write_485DR@CMemRegpcie950@@UAEXE@Z 10006ac2 f i pddpcie950:pddpcie950.obj
 0001:00005ada       ?Read_485DR@CMemRegpcie950@@UAEEXZ 10006ada f i pddpcie950:pddpcie950.obj
 0001:00005ae9       ?Read_ID1@CMemRegpcie950@@UAEEXZ 10006ae9 f i pddpcie950:pddpcie950.obj
 0001:00005af8       ?Read_ID2@CMemRegpcie950@@UAEEXZ 10006af8 f i pddpcie950:pddpcie950.obj
 0001:00005b07       ?Read_ID3@CMemRegpcie950@@UAEEXZ 10006b07 f i pddpcie950:pddpcie950.obj
 0001:00005b16       ?WRITE_550_REGISTER@CMemRegpcie950@@UAEXPAEE@Z 10006b16 f i pddpcie950:pddpcie950.obj
 0001:00005b54       ?READ_550_REGISTER@CMemRegpcie950@@UAEEPAE@Z 10006b54 f i pddpcie950:pddpcie950.obj
 0001:00005b95       ?WRITE_650_REGISTER@CMemRegpcie950@@UAEXPAEE@Z 10006b95 f i pddpcie950:pddpcie950.obj
 0001:00005b95       ?WRITE_950_REGISTER@CMemRegpcie950@@UAEXPAEE@Z 10006b95 f i pddpcie950:pddpcie950.obj
 0001:00005b95       ?WRITE_ICR_REGISTER@CMemRegpcie950@@UAEXPAEE@Z 10006b95 f i pddpcie950:pddpcie950.obj
 0001:00005ba9       ?READ_ICR_REGISTER@CMemRegpcie950@@UAEEPAE@Z 10006ba9 f i pddpcie950:pddpcie950.obj
 0001:00005ba9       ?READ_950_REGISTER@CMemRegpcie950@@UAEEPAE@Z 10006ba9 f i pddpcie950:pddpcie950.obj
 0001:00005ba9       ?READ_650_REGISTER@CMemRegpcie950@@UAEEPAE@Z 10006ba9 f i pddpcie950:pddpcie950.obj
 0001:00005bb9       ??_ECRegpcie950@@UAEPAXI@Z 10006bb9 f i pddpcie950:pddpcie950.obj
 0001:00005bb9       ??_GCMemRegpcie950@@UAEPAXI@Z 10006bb9 f i pddpcie950:pddpcie950.obj
 0001:00005bb9       ??_ECMemRegpcie950@@UAEPAXI@Z 10006bb9 f i pddpcie950:pddpcie950.obj
 0001:00005bb9       ??_GCRegpcie950@@UAEPAXI@Z 10006bb9 f i pddpcie950:pddpcie950.obj
 0001:00005bd8       ??0CPddpcie950@@QAE@PAGPAXPAU__HWOBJ@@@Z 10006bd8 f   pddpcie950:pddpcie950.obj
 0001:00005c76       ?SerialRegisterBackup@CPddpcie950@@UAEXXZ 10006c76 f i pddpcie950:pddpcie950.obj
 0001:00005c84       ?SerialRegisterRestore@CPddpcie950@@UAEXXZ 10006c84 f i pddpcie950:pddpcie950.obj
 0001:00005c92       ?ModemInterruptHandler@CPddpcie950@@UAEXXZ 10006c92 f i pddpcie950:pddpcie950.obj
 0001:00005c9a       ?GetRxBufferSize@CPddpcie950@@UAEKXZ 10006c9a f i pddpcie950:pddpcie950.obj
 0001:00005c9d       ?LineInterruptHandler@CPddpcie950@@UAEXXZ 10006c9d f i pddpcie950:pddpcie950.obj
 0001:00005ca2       ??1CPddpcie950@@UAE@XZ     10006ca2 f   pddpcie950:pddpcie950.obj
 0001:00005d92       ?CreateHardwareAccess@CPddpcie950@@UAEHXZ 10006d92 f   pddpcie950:pddpcie950.obj
 0001:00005e36       ?XmitInterruptHandler@CPddpcie950@@UAEXPAEPAK@Z 10006e36 f   pddpcie950:pddpcie950.obj
 0001:00005ee3       ??_GCPddpcie950@@UAEPAXI@Z 10006ee3 f i pddpcie950:pddpcie950.obj
 0001:00005ee3       ??_ECPddpcie950@@UAEPAXI@Z 10006ee3 f i pddpcie950:pddpcie950.obj
 0001:00005f02       ?GetIsrInfo@CRegistryEdit@@QAEKPAU_DDKISRINFO_tag@@@Z 10006f02 f i pddpcie950:pddisrpcie950.obj
 0001:00005f2a       ??0CPddpcie950Isr@@QAE@PAGPAXPAU__HWOBJ@@@Z 10006f2a f   pddpcie950:pddisrpcie950.obj
 0001:00005f75       ??1CPddpcie950Isr@@UAE@XZ  10006f75 f   pddpcie950:pddisrpcie950.obj
 0001:00005fdd       ?Init@CPddpcie950Isr@@UAEHXZ 10006fdd f   pddpcie950:pddisrpcie950.obj
 0001:000063b7       ?PeekEventData@CPddpcie950Isr@@IAEHPAE0@Z 100073b7 f i pddpcie950:pddisrpcie950.obj
 0001:00006434       ?ReadEventData@CPddpcie950Isr@@IAEHPAE0@Z 10007434 f i pddpcie950:pddisrpcie950.obj
 0001:00006484       ?EmptyEventData@CPddpcie950Isr@@UAEXXZ 10007484 f   pddpcie950:pddisrpcie950.obj
 0001:000064b3       ?WriteXmitData@CPddpcie950Isr@@IAEHE@Z 100074b3 f i pddpcie950:pddisrpcie950.obj
 0001:0000651b       ?ThreadRun@CPddpcie950Isr@@EAEKXZ 1000751b f   pddpcie950:pddisrpcie950.obj
 0001:0000662b       ?ReceiveInterruptHandler@CPddpcie950Isr@@UAEKPAEPAK@Z 1000762b f   pddpcie950:pddisrpcie950.obj
 0001:000067e3       ?CancelReceive@CPddpcie950Isr@@UAEKXZ 100077e3 f   pddpcie950:pddisrpcie950.obj
 0001:00006838       ?FilterFunction@@YAHK@Z    10007838 f   pddpcie950:pddisrpcie950.obj
 0001:00006863       ?XmitInterruptHandler@CPddpcie950Isr@@UAEXPAEPAK@Z 10007863 f   pddpcie950:pddisrpcie950.obj
 0001:00006b14       ?XmitComChar@CPddpcie950Isr@@UAEXE@Z 10007b14 f   pddpcie950:pddisrpcie950.obj
 0001:00006c35       ?CancelXmit@CPddpcie950Isr@@UAEHXZ 10007c35 f   pddpcie950:pddisrpcie950.obj
 0001:00006c91       ?LineInterruptHandler@CPddpcie950Isr@@UAEXXZ 10007c91 f   pddpcie950:pddisrpcie950.obj
 0001:00006cf0       ?ModemInterruptHandler@CPddpcie950Isr@@UAEXXZ 10007cf0 f   pddpcie950:pddisrpcie950.obj
 0001:00006d47       ?GetRxBufferSize@CPddpcie950Isr@@UAEKXZ 10007d47 f   pddpcie950:pddisrpcie950.obj
 0001:00006d54       ??_GCPddpcie950Isr@@UAEPAXI@Z 10007d54 f i pddpcie950:pddisrpcie950.obj
 0001:00006d54       ??_ECPddpcie950Isr@@UAEPAXI@Z 10007d54 f i pddpcie950:pddisrpcie950.obj
 0001:00006d74       _CreateBusAccessHandle     10007d74 f   ceddk:CEDDK.dll
 0001:00006d7a       _DDKPwr_RequestLevel       10007d7a f   ceddk:CEDDK.dll
 0001:00006d80       _DDKPwr_ReleaseLevel       10007d80 f   ceddk:CEDDK.dll
 0001:00006d86       _SetDevicePowerState       10007d86 f   ceddk:CEDDK.dll
 0001:00006d8c       _DDKPwr_Initialize         10007d8c f   ceddk:CEDDK.dll
 0001:00006d92       _DDKPwr_Deinitialize       10007d92 f   ceddk:CEDDK.dll
 0001:00006d98       _CloseBusAccessHandle      10007d98 f   ceddk:CEDDK.dll
 0001:00006d9e       _WRITE_PORT_UCHAR          10007d9e f   ceddk:CEDDK.dll
 0001:00006da4       _READ_PORT_UCHAR           10007da4 f   ceddk:CEDDK.dll
 0001:00006daa       _MmMapIoSpace              10007daa f   ceddk:CEDDK.dll
 0001:00006db0       _TranslateBusAddr          10007db0 f   ceddk:CEDDK.dll
 0001:00006db6       _WRITE_REGISTER_UCHAR      10007db6 f   ceddk:CEDDK.dll
 0001:00006dbc       _READ_REGISTER_UCHAR       10007dbc f   ceddk:CEDDK.dll
 0001:00006dc2       _MmUnmapIoSpace            10007dc2 f   ceddk:CEDDK.dll
 0001:00006dc8       _HalFreeCommonBuffer       10007dc8 f   ceddk:CEDDK.dll
 0001:00006dce       _BusTransBusAddrToStatic   10007dce f   ceddk:CEDDK.dll
 0001:00006dd4       _HalAllocateCommonBuffer   10007dd4 f   ceddk:CEDDK.dll
 0001:00006dda       _EventModify               10007dda f   coredll:COREDLL.dll
 0001:00006de0       _DisableThreadLibraryCalls 10007de0 f   coredll:COREDLL.dll
 0001:00006de6       _LeaveCriticalSection      10007de6 f   coredll:COREDLL.dll
 0001:00006dec       _SetProcPermissions        10007dec f   coredll:COREDLL.dll
 0001:00006df2       _EnterCriticalSection      10007df2 f   coredll:COREDLL.dll
 0001:00006df8       _InterruptDisable          10007df8 f   coredll:COREDLL.dll
 0001:00006dfe       _InterruptDone             10007dfe f   coredll:COREDLL.dll
 0001:00006e04       _LocalFree                 10007e04 f   coredll:COREDLL.dll
 0001:00006e0a       _DeleteCriticalSection     10007e0a f   coredll:COREDLL.dll
 0001:00006e10       _ExitThread                10007e10 f   coredll:COREDLL.dll
 0001:00006e16       _CreateThread              10007e16 f   coredll:COREDLL.dll
 0001:00006e1c       _InterruptInitialize       10007e1c f   coredll:COREDLL.dll
 0001:00006e22       _OpenDeviceKey             10007e22 f   coredll:COREDLL.dll
 0001:00006e28       _InitializeCriticalSection 10007e28 f   coredll:COREDLL.dll
 0001:00006e2e       _LocalAlloc                10007e2e f   coredll:COREDLL.dll
 0001:00006e34       _CeFreeAsynchronousBuffer  10007e34 f   coredll:COREDLL.dll
 0001:00006e3a       _CeAllocAsynchronousBuffer 10007e3a f   coredll:COREDLL.dll
 0001:00006e40       _TerminateThread           10007e40 f   coredll:COREDLL.dll
 0001:00006e46       _SetInterruptEvent         10007e46 f   coredll:COREDLL.dll
 0001:00006e4c       _CeEventHasOccurred        10007e4c f   coredll:COREDLL.dll
 0001:00006e52       _DDKReg_GetWindowInfo      10007e52 f   coredll:COREDLL.dll
 0001:00006e58       _InterruptMask             10007e58 f   coredll:COREDLL.dll
 0001:00006e5e       _CharUpperW                10007e5e f   coredll:COREDLL.dll
 0001:00006e64       _DDKReg_GetIsrInfo         10007e64 f   coredll:COREDLL.dll
 0001:00006e6a       _KernelLibIoControl        10007e6a f   coredll:COREDLL.dll
 0001:00006e70       _FreePhysMem               10007e70 f   coredll:COREDLL.dll
 0001:00006e76       _NKDbgPrintfW              10007e76 f   coredll:COREDLL.dll
 0001:00006e7c       _DllMain                   10007e7c f   corelib0:dllmain.obj
 0001:00006f3b       __DllMainCRTStartup        10007f3b f   corelib0:pegdmain.obj
 0001:00006f4f       ___security_init_cookie    10007f4f f   corelib0:seccinit.obj
 0001:00006f7a       @__security_check_cookie@4 10007f7a f   corelib0:x86secgs.obj
 0001:00006fa0       __SEH_prolog4              10007fa0 f   corelib0:sehprolg4.obj
 0001:00006fe5       __SEH_epilog4              10007fe5 f   corelib0:sehprolg4.obj
 0001:00006ff9       __except_handler4          10007ff9 f   corelib0:chandler4gs.obj
 0001:0000709e       __cexit                    1000809e f   corelib0:cexit.obj
 0001:000070af       __initterm                 100080af f   corelib0:crt0dat.obj
 0001:000070cb       __cinit                    100080cb f   corelib0:crt0dat.obj
 0001:000070ee       ??2@YAPAXI@Z               100080ee f   corelib1:COREDLL.dll
 0001:000070f4       _memcpy                    100080f4 f   corelib1:COREDLL.dll
 0001:000070fa       _memset                    100080fa f   corelib1:COREDLL.dll
 0001:00007100       __purecall                 10008100 f   corelib1:COREDLL.dll
 0001:00007106       ??3@YAXPAX@Z               10008106 f   corelib1:COREDLL.dll
 0001:0000710c       _wcsrchr                   1000810c f   corelib1:COREDLL.dll
 0001:00007112       _wcsstr                    10008112 f   corelib1:COREDLL.dll
 0001:00007118       _wcstoul                   10008118 f   corelib1:COREDLL.dll
 0001:0000711e       __ultow                    1000811e f   corelib1:COREDLL.dll
 0001:00007124       _wcsncpy                   10008124 f   corelib1:COREDLL.dll
 0001:0000712a       _memchr                    1000812a f   corelib1:COREDLL.dll
 0001:00007130       __XcptFilter               10008130 f   corelib1:COREDLL.dll
 0001:00007136       ___security_gen_cookie2    10008136 f   corelib1:COREDLL.dll
 0001:0000713c       ___report_gsfailure        1000813c f   corelib1:COREDLL.dll
 0001:00007142       __except_handler4_common   10008142 f   corelib1:COREDLL.dll
 0001:00007148       _free                      10008148 f   corelib1:COREDLL.dll
 0001:0000714e       _TerminateProcess          1000814e f   coredll:COREDLL.dll
 0001:00007194       __IMPORT_DESCRIPTOR_CEDDK  10008194     ceddk:CEDDK.dll
 0001:000071a8       __IMPORT_DESCRIPTOR_COREDLL 100081a8     coredll:COREDLL.dll
 0001:000071bc       __NULL_IMPORT_DESCRIPTOR   100081bc     ceddk:CEDDK.dll
 0002:00000000       __imp__CreateBusAccessHandle 10009000     ceddk:CEDDK.dll
 0002:00000004       __imp__DDKPwr_RequestLevel 10009004     ceddk:CEDDK.dll
 0002:00000008       __imp__DDKPwr_ReleaseLevel 10009008     ceddk:CEDDK.dll
 0002:0000000c       __imp__SetDevicePowerState 1000900c     ceddk:CEDDK.dll
 0002:00000010       __imp__DDKPwr_Initialize   10009010     ceddk:CEDDK.dll
 0002:00000014       __imp__DDKPwr_Deinitialize 10009014     ceddk:CEDDK.dll
 0002:00000018       __imp__CloseBusAccessHandle 10009018     ceddk:CEDDK.dll
 0002:0000001c       __imp__WRITE_PORT_UCHAR    1000901c     ceddk:CEDDK.dll
 0002:00000020       __imp__READ_PORT_UCHAR     10009020     ceddk:CEDDK.dll
 0002:00000024       __imp__MmMapIoSpace        10009024     ceddk:CEDDK.dll
 0002:00000028       __imp__TranslateBusAddr    10009028     ceddk:CEDDK.dll
 0002:0000002c       __imp__WRITE_REGISTER_UCHAR 1000902c     ceddk:CEDDK.dll
 0002:00000030       __imp__READ_REGISTER_UCHAR 10009030     ceddk:CEDDK.dll
 0002:00000034       __imp__MmUnmapIoSpace      10009034     ceddk:CEDDK.dll
 0002:00000038       __imp__HalFreeCommonBuffer 10009038     ceddk:CEDDK.dll
 0002:0000003c       __imp__BusTransBusAddrToStatic 1000903c     ceddk:CEDDK.dll
 0002:00000040       __imp__HalAllocateCommonBuffer 10009040     ceddk:CEDDK.dll
 0002:00000044       \177CEDDK_NULL_THUNK_DATA  10009044     ceddk:CEDDK.dll
 0002:00000048       __imp__EventModify         10009048     coredll:COREDLL.dll
 0002:0000004c       __imp__DisableThreadLibraryCalls 1000904c     coredll:COREDLL.dll
 0002:00000050       __imp__LeaveCriticalSection 10009050     coredll:COREDLL.dll
 0002:00000054       __imp__SetProcPermissions  10009054     coredll:COREDLL.dll
 0002:00000058       __imp__EnterCriticalSection 10009058     coredll:COREDLL.dll
 0002:0000005c       __imp__InterruptDisable    1000905c     coredll:COREDLL.dll
 0002:00000060       __imp__InterruptDone       10009060     coredll:COREDLL.dll
 0002:00000064       __imp__CloseHandle         10009064     coredll:COREDLL.dll
 0002:00000068       __imp__Sleep               10009068     coredll:COREDLL.dll
 0002:0000006c       __imp__WaitForSingleObject 1000906c     coredll:COREDLL.dll
 0002:00000070       __imp__CeSetThreadPriority 10009070     coredll:COREDLL.dll
 0002:00000074       __imp__CeGetThreadPriority 10009074     coredll:COREDLL.dll
 0002:00000078       __imp__SetLastError        10009078     coredll:COREDLL.dll
 0002:0000007c       __imp__SetThreadPriority   1000907c     coredll:COREDLL.dll
 0002:00000080       __imp__LocalFree           10009080     coredll:COREDLL.dll
 0002:00000084       __imp__DeleteCriticalSection 10009084     coredll:COREDLL.dll
 0002:00000088       __imp__GetTickCount        10009088     coredll:COREDLL.dll
 0002:0000008c       __imp__ExitThread          1000908c     coredll:COREDLL.dll
 0002:00000090       __imp__CreateThread        10009090     coredll:COREDLL.dll
 0002:00000094       __imp__InterruptInitialize 10009094     coredll:COREDLL.dll
 0002:00000098       __imp__RegCloseKey         10009098     coredll:COREDLL.dll
 0002:0000009c       __imp__RegQueryValueExW    1000909c     coredll:COREDLL.dll
 0002:000000a0       __imp__OpenDeviceKey       100090a0     coredll:COREDLL.dll
 0002:000000a4       __imp__CreateEventW        100090a4     coredll:COREDLL.dll
 0002:000000a8       __imp__InitializeCriticalSection 100090a8     coredll:COREDLL.dll
 0002:000000ac       __imp__LocalAlloc          100090ac     coredll:COREDLL.dll
 0002:000000b0       __imp__CeFreeAsynchronousBuffer 100090b0     coredll:COREDLL.dll
 0002:000000b4       __imp__CeAllocAsynchronousBuffer 100090b4     coredll:COREDLL.dll
 0002:000000b8       __imp__ResumeThread        100090b8     coredll:COREDLL.dll
 0002:000000bc       __imp__TerminateThread     100090bc     coredll:COREDLL.dll
 0002:000000c0       __imp__SetInterruptEvent   100090c0     coredll:COREDLL.dll
 0002:000000c4       __imp__RegOpenKeyExW       100090c4     coredll:COREDLL.dll
 0002:000000c8       __imp__CeEventHasOccurred  100090c8     coredll:COREDLL.dll
 0002:000000cc       __imp__DDKReg_GetWindowInfo 100090cc     coredll:COREDLL.dll
 0002:000000d0       __imp__InterruptMask       100090d0     coredll:COREDLL.dll
 0002:000000d4       __imp__RegSetValueExW      100090d4     coredll:COREDLL.dll
 0002:000000d8       __imp__CharUpperW          100090d8     coredll:COREDLL.dll
 0002:000000dc       __imp__DDKReg_GetIsrInfo   100090dc     coredll:COREDLL.dll
 0002:000000e0       __imp__KernelLibIoControl  100090e0     coredll:COREDLL.dll
 0002:000000e4       __imp__FreePhysMem         100090e4     coredll:COREDLL.dll
 0002:000000e8       __imp__NKDbgPrintfW        100090e8     coredll:COREDLL.dll
 0002:000000ec       __imp_??2@YAPAXI@Z         100090ec     corelib1:COREDLL.dll
 0002:000000f0       __imp__memcpy              100090f0     corelib1:COREDLL.dll
 0002:000000f4       __imp__memset              100090f4     corelib1:COREDLL.dll
 0002:000000f8       __imp___purecall           100090f8     corelib1:COREDLL.dll
 0002:000000fc       __imp_??3@YAXPAX@Z         100090fc     corelib1:COREDLL.dll
 0002:00000100       __imp__wcsrchr             10009100     corelib1:COREDLL.dll
 0002:00000104       __imp__wcsstr              10009104     corelib1:COREDLL.dll
 0002:00000108       __imp__wcstoul             10009108     corelib1:COREDLL.dll
 0002:0000010c       __imp___ultow              1000910c     corelib1:COREDLL.dll
 0002:00000110       __imp__wcsncpy             10009110     corelib1:COREDLL.dll
 0002:00000114       __imp__memchr              10009114     corelib1:COREDLL.dll
 0002:00000118       __imp___XcptFilter         10009118     corelib1:COREDLL.dll
 0002:0000011c       __imp____security_gen_cookie2 1000911c     corelib1:COREDLL.dll
 0002:00000120       __imp____report_gsfailure  10009120     corelib1:COREDLL.dll
 0002:00000124       __imp___except_handler4_common 10009124     corelib1:COREDLL.dll
 0002:00000128       __imp__free                10009128     corelib1:COREDLL.dll
 0002:0000012c       __imp__TerminateProcess    1000912c     coredll:COREDLL.dll
 0002:00000130       \177COREDLL_NULL_THUNK_DATA 10009130     coredll:COREDLL.dll
 0002:00000154       ___security_cookie         10009154     corelib0:seccinit.obj
 0002:00000158       ___security_cookie_complement 10009158     corelib0:seccinit.obj
 0002:00000170       __exitflag                 10009170     corelib0:cexit.obj
 0002:00000174       ___onexitend               10009174     <common>
 0002:00000178       ___onexitbegin             10009178     <common>
 0002:0000017c       __pRawDllMain              1000917c     <common>

 entry point at        0001:00006f3b

 Static symbols

 0001:00001c48       ?SerialDispatchThread@@YAKPAX@Z 10002c48 f   mddpcie950:mddpcie950.obj
 0001:00006e93       __DllMainCRTStartupHelper  10007e93 f   corelib0:pegdmain.obj
 0001:0000701c       _doexit                    1000801c f   corelib0:cexit.obj
